:10000000E8890010250100002D0100002F010000EB
:10001000310100003301000035010000FE6EFFEFEA
:100020000000000000000000000000003701000098
:1000300039010000000000003B0100009D010000AC
:100040003F010000490100003F0100003F010000A6
:100050003F0100003F0100003F0100003F010000A0
:100060003F0100003F0100003F0100003F01000090
:100070003F010000000000003F0100003F010000C0
:100080003F0100003F0100003F0100003F01000070
:100090003F0100003F0100003F0100003F01000060
:1000A000932400003F0100003F0100003F010000D9
:1000B0003F0100003F0100003F0100003F01000040
:1000C0003F0100003F0100003F0100003F01000030
:1000D0003F0100003F0100003F0100003F01000020
:1000E0003F010000DFF80CD000F054F90048004751
:1000F0001D090000E8890010D0F800D0D0F804F005
:10010000024600200B21C30700D0802303EB5000E0
:1001100012F8013B491E184409B2C0B20029F2D1BD
:10012000704700000648804706480047FEE7FEE7A4
:10013000FEE7FEE7FEE7FEE7FEE7FEE7FEE7FEE797
:10014000A3170000E500000010B54FF0402101208A
:10015000086001F06CFD10BD10B54FF0E0241A48A6
:1001600060611F21601700F01EF80020A0610720C9
:10017000206110BD154810B50221416000210167C2
:1001800041611D22C260C16301214160FFF7E4FFAC
:100190000221C81E00F007F8002010BD0C480168BD
:1001A000491C01607047C906090E002806DA00F0F4
:1001B0000F0000F1E02080F8141D704700F1E020EE
:1001C00080F8001470470000BFD40100000009400F
:1001D0008401001010B50B4604461146184600F085
:1001E000C5F8C4E9000110BD02E008C8121F08C12B
:1001F000002AFAD1704770470000000044332211F2
:1002000070B5284C607820B30026274D012810D007
:1002100002280DD1A8686168401A2449884215D384
:100220002348406B400011D5012002F008F86670A9
:1002300070BDA8686168401A1E498842F8D3002042
:1002400001F0FDFFA86860600220607026700C203D
:1002500005E020780028EBD1012020700D20BDE8BA
:10026000704001F087B9002802D10E490120487082
:10027000704710B501F000FD0A490020487010BD1C
:1002800008480121417008498968416070477047FA
:100290007047022803D0032803D100F0EFBE00F01E
:1002A0000ABF7047B401001000000940A086010099
:1002B0000080092040420F0040EA01039B0703D061
:1002C00009E008C9121F08C0042AFAD203E011F895
:1002D000013B00F8013B521EF9D27047002001E0BB
:1002E00001C1121F002AFBD170471201100100004A
:1002F000004051C20313000104204801FFFFFFFF2B
:100300001948062101610721016000214161416214
:1003100002214160C168C906FCD400E08168C1685F
:100320004907FBD4002070470F498860C868C006A1
:10033000FCD48868704700B50B46024604E000BF55
:1003400012F8010BFFF7F0FF5B1EF9D200BD00B5FC
:100350000B46024604E00020FFF7E6FF02F8010B1F
:100360005B1EF8D200BD00000000034070B5002401
:100370002546002801DA01244042002901DA01253E
:10038000494200F019F8AC4200D04042002C00D0A5
:10039000494270BD064C074D06E0E06840F001039D
:1003A00094E8070098471034AC42F6D3FFF79EFE5E
:1003B000E40300000404000030B50B4601460020B1
:1003C0002022012409E021FA02F59D4205D303FA17
:1003D00002F5491B04FA02F52844151EA2F1010298
:1003E000F1DC30BD5434000000000010C8010000F2
:1003F000DC300000FC340000C80100102088000040
:10040000DC020000CF06000010B50178427801EB55
:10041000810102EB4101C902A1F5C0318AB2C17864
:100420000479303901EB810104EB41014901A1F567
:10043000C06101F4FC611143C27980796FF02F0330
:10044000303800EB800003EB40001044C0F3440060
:10045000084310BDF0B58DB004463022F649684619
:10046000FFF72AFFE079A17A00EB4002C2EBC0104F
:1004700001EBC000217A642211FB02F1627A1023A1
:1004800002EB820201EB420108444002742100EBBE
:1004900041202179627901EB810103EB4101114493
:1004A00080B201F01F010143237800204FEA0D05BF
:1004B00055F820201678B3420DD166785778BE42A1
:1004C00009D1A6789278964205D14001203000F4F7
:1004D000F070014303E0401CC0B20C28E8D30DB01B
:1004E0000846F0BDD54910B5486980040CD4D44AFB
:1004F000906843F698239468241A9C42FBD3486979
:10050000800401D4012010BD052001F033F8002043
:1005100010BD70B5CA4CA668042001F02BF8C94D77
:1005200003E000BFFFF7DEFF48B1A068801BA842D0
:10053000F8D308E0FFF7D6FF08B1012070BDA0682E
:10054000801BA842F6D3002070BD10B5092001F031
:1005500011F8BD490120487010BD2DE9F04100257A
:1005600006462C46B94F0BE040222146B74800F022
:10057000E2FE00203958001D0D444028FAD34034D3
:10058000B442F1D32846BDE8F081B1A386B00FCBC9
:100590008DE80F00B2A0B3490068049008680026F7
:1005A0004FF6FF021040B04A40F4807010430860DC
:1005B000AE49AF4F4FF4F4200E60AF493860AD48FC
:1005C0000860AE494012AE4D0860F8202870FF2048
:1005D0006870A870AB48B046D0F8189001F0A2FA45
:1005E000994CDFF8A4A24FF0010B606801280FD1ED
:1005F0004FF4F420FFF7B1FFE0B3D4F8042020203B
:100600004346514651F822703B54401C4028F9D3D0
:10061000616800205AF821102B180A5C401C83F8EE
:1006200000246028F8D301F049FE012001F007FE04
:100630004FF4E17A5546514640F2491001F0D7FA9D
:10064000294640F29F1001F0D2FAA046FFF7D8FDEC
:1006500098F8010045460028F8D100218BA000F051
:1006600076FD0400F2D08A48017A66297DD04629B9
:100670007BD0DDE0FFE784F800B003223B68022175
:10068000104601EB932740F6FF7E13E0B0EB932F6B
:1006900001D3714600E0411CC0F3032C4CEA011861
:1006A000A85405EB020C09098CF80180801C8CF819
:1006B0000210D21C8742E9D8402240F2044163482C
:1006C00000F039FE61498878032802D3584681F842
:1006D00002B0C0B204AA5746125C60685AF82030D3
:1006E00083F843205AF8203083F827204B786A4655
:1006F00002EB13135AF820C01B788CF844305AF8D8
:1007000020C08CF829304B7857F820C003F00F0335
:100710001DF803308CF8453057F820C08CF82E3087
:100720000B7857F820C002EB13131B788CF8463077
:1007300057F820C08CF83030097801F00F01515C77
:1007400057F8202082F8471057F8202082F83210FE
:1007500057F820004030FFF7D3FC616857F82110AC
:1007600081F82D0039480C3000E01CE0FFF772FEE4
:10077000616857F82120A2F8580057F82120A2F804
:10078000520057F82110A1F8500030481C30FFF7F4
:100790003BFE616857F82120A2F8560057F8211057
:1007A000A1F84E0034E7417A722905D0522903D0CE
:1007B000642901D044293BD1817A6D2906D04D2985
:1007C00004D0782901D0582932D101263048007848
:1007D000662801D046282BD1402211011B4800F089
:1007E000AAFD012E03D14021184800F0AFFD1749A2
:1007F00027480F7B001D091D00F04DFDC0B1686842
:10080000A84628B14FF4F420FFF7A7FE98B10FE0F7
:1008100038461F4900F018FD50B10C481C49007AB9
:1008200000F01EFD20B14FF4F420FFF796FE88B3D0
:10083000FFF78BFE0AE760E03032000000800920FD
:100840000000094080841E00C8000010C807001086
:1008500030313233343536373839414243444546F6
:10086000454E46000CED00E00000FA0510010010B6
:100870000001001000BC0700F8000010FC00001090
:10088000C801001060320000C00000104634320081
:1008900074080010FFE70A2000F06CFE00273D46B8
:1008A000072000F067FE0FE0A8050DD1204600F0FC
:1008B00028FC0446A0F57060FF381ED0032C1CD322
:1008C00040F6F870844218D2402229464A4800F087
:1008D00032FD4035012E03D14021474800F036FD5E
:1008E00009EB07004022444900F0B0FD07204037E3
:1008F00000F040FE002DE7D0D6E70B2000F03AFED6
:100900005446514640F29F1001F071F9214640F2E1
:10091000491001F06CF988F801B097E600F041FF4A
:1009200000F096FFFFF726FC00F0EAFD002000F043
:1009300021FEFFF7E5FC314E7069314D314CDFF897
:10094000C88040034FF0000702D5FFF7CBFD88B306
:10095000042000F00FFE7069800414D4FFF7D9FD65
:1009600040B3FFF7D6FD28B3FFF7D3FD10B3042043
:1009700000F000FEA06841467269920403D4A268A8
:10098000121A8A42F8D3A06842F21071A268121AB1
:100990008A42FBD3706B10F0004F17D5706D0006C4
:1009A00014D50120686000F098FC4FF4F420FFF7A4
:1009B000D4FD58B100F07EFD00284FF002000AD0AF
:1009C00000F0D8FD6868401C02D00AE06F60F1E7D3
:1009D00000F06AFD05E000F0CDFD6868401C00D124
:1009E0006F6000F07AFCA0684146A268121A8A4241
:1009F000FBD3FFF7CAFD0000C807001000800920E4
:100A0000C80000100000094080841E002DE9F84352
:100A100000250E460446FE4FA84634E0B4F5007F9C
:100A200019D2132C0DD0142C0ED0B4F5FF7F0ED09C
:100A3000A4F58070FF380CD03E2C1CD8F548005D22
:100A400012E097F820000FE0388C000A0CE05520E7
:100A50000AE0AA2008E0B4F5006F08D2EE4820446E
:100A6000A0F5805090F8000E8DF8000005E0EB48EE
:100A7000006801280BD08DF80080E9499DF800003E
:100A8000641C48556D1CB542C8D3BDE8F8830122EB
:100A9000A4F50061684600F04EFCEEE770B5DC4D51
:100AA0002C6B402C00D94024E86AE96902198A427B
:100AB00002D90C1A042169702146FFF7A7FF2246CC
:100AC000D749822001F0BBFCE86A2044E862286B29
:100AD000011BD348296300F19F008268A2EB040246
:100AE000826005D06978022901D00021017370BDB0
:100AF00003216970F9E7CA4910B59F31C9480860F8
:100B00000D22822001F09BFCC1490520487010BDD8
:100B100070B50D46C4494A69520302D5496D49056D
:100B200021D4B0F5007F1ED3C04BB94CB0F5006F97
:100B30001AD29968A269891ABD4A914204D3996868
:100B4000A161002161606161B54A00214032B24B70
:100B500007E044181C44565CA4F58054491C84F8F2
:100B6000006EA942F5D370BD616921B99968A16190
:100B700099686161A060A949096829B10129F2D188
:100B8000AC4909780029EED199686269891AAA4AA4
:100B9000914217D29968A16199686161A168401A70
:100BA0006168884203D9616A884200D26060062089
:100BB00000F0E0FC2A466168BDE87040984840308B
:100BC00000F0A7BBBDE870400C2000F0D3BC10B50E
:100BD0008F4CA178E06A4218E1698A4206D9081A66
:100BE000A07005206070022001F0E4FBA178E06AAB
:100BF000FFF78EFFA178E06A0844E062206B421A9A
:100C00008748226300F19F008368A3EB01018160A4
:100C100002D06178052904D100210173BDE810409C
:100C200069E710BD2DE9F041794CA178E06A4218DE
:100C3000E1698A4206D9081AA07005206070022076
:100C400001F0B8FB764B0021A07803F14005E26A81
:100C500008E056186F5C9E5DBE4202D00021A16282
:100C600002E0491C8142F4D31118E162216B0A1A97
:100C70006B49226301F19F018B68A3EB0000886040
:100C800002D06078052808D1A06A20B1002008733E
:100C9000BDE8F0412FE70120F9E7BDE8F0816048A9
:100CA00010B58030D0F81110027D09BA21F0FF0193
:100CB0001143574A4902D162C18A49BA49021163B4
:100CC000806888420DD0822001F074FB022001F080
:100CD00071FB534902209F310873FFF70CFF00207E
:100CE00010BD012010BD70B54D48803002248168D0
:100CF00000F11F0529B1007B000607D4022001F096
:100D000059FB2C73FFF7F7FE002070BD012070BD6A
:100D100010B543483E4C80308068A178884200D2AC
:100D2000A0703F49A2784031822001F088FB032067
:100D300060703B48A2789F308168891A81600021E9
:100D4000017310BD364810B58030816839B1007B21
:100D5000000601D5822000E0022001F02BFB304983
:100D600000209F310873BDE81040C4E610B5FFF7BE
:100D7000BAFF00281FD02A4870214030022201709B
:100D8000002141708270C1700171417181710A222C
:100D9000C271017241728172C172302202730122EA
:100DA00042738173C17301744174194912208870B0
:100DB000BDE81040ACE710BD1CB5FFF794FF00285C
:100DC00068D01E480A2206210388684600F020FAEF
:100DD000134800224030802302704370827001214A
:100DE000C1702021017143718271C271412202726E
:100DF000542242724F2282724C22C272017341739A
:100E00008173C1734622027450234374722317E026
:100E1000DC000010F0310000C8010010CC00001010
:100E2000C8070010555342530080092000000940B4
:100E3000A0860100C800001020A1070004040000E3
:100E400083746923C3746E2303757423437581759A
:100E5000C2756C2202766122427673228276682203
:100E6000C276017741778177C1779DF8011080F8CC
:100E700020109DF8021080F821109DF8031080F8D2
:100E800022109DF8041080F82310DD49242088707A
:100E9000FFF73EFF1CBD10B5FFF725FF00280CD063
:100EA000D84803210170002141708170C170D4497C
:100EB00004208870BDE810402AE710BD10B5FFF788
:100EC00012FF002810D0CF48002106220170427086
:100ED0008170C170017141718171C171C84908206F
:100EE0008870BDE8104013E710BD10B5FFF7FBFE9A
:100EF000002815D0C24AC348116A491E0B0E037060
:100F00000B0C43700B0A8370C17000210171417199
:100F100002238371C17108209070BDE81040F7E68C
:100F200010BD10B5FFF7DFFE002819D0B54800212D
:100F3000B34B0170417081700822C2701A6A140E9E
:100F40000471140C4471140A8471C2710222027279
:100F500041728272C1720C209870BDE81040D7E6D1
:100F600010BD2DE9F041A64DA64C0021A8784034D3
:100F7000A44A02E0535C6354491C03468142F9D3FE
:100F80001F2B72D12068A04988426ED19D4E6068A7
:100F90005F364FF001087060A068B060607B18B9E0
:100FA000A07B08B1102802D986F80C8059E0E07BBC
:100FB0001E28F9D00FDC12282ED005DC48B30328F8
:100FC000F2D1BDE8F041D1E61528EDD01A28EBD1D9
:100FD000BDE8F0415FE702272A2828D010DC23284B
:100FE0001DD025281ED02828DED1FFF758FE002866
:100FF00026D0207B000618D56F70BDE8F0414DE586
:101000002F281ED05528CFD05A28CDD1BDE8F04189
:1010100054E7BDE8F04195E6BDE8F041CCE6BDE817
:10102000F0417EE7BDE8F0415FE7022016E0FFF700
:1010300036FE002804D0207B00060ED485F80180FF
:101040002BE6FFF72CFE0028FAD0207B000604D404
:1010500085F80180C5F828801FE6822001F0AAF9F2
:101060003773BDE8F04146E5FFE7822001F0A2F9C1
:10107000022001F09FF9062068700EE6604810B566
:101080004178022908D003290ED004290FD0052960
:1010900001D10021417010BD5A484030C07B282842
:1010A000F9D1BDE81040F9E4BDE8104023E5822005
:1010B00001F080F9F8E710B55249022001F08EF9ED
:1010C0004F498870487858B101280CD0022001F0AF
:1010D00071F94C4902205F310873BDE810400AE500
:1010E000BDE810403DE747484030C07B2A2804D087
:1010F0002F2805D1BDE8104094E5BDE8104066E515
:1011000010BDFFB50246002002EB420501464FF438
:1011100000666C4603AA6B1844F82130B34202DD26
:10112000002004B0F0BD394F07EB6307DB073F78C1
:10113000575401D03B095354535C8F0003F00F0305
:101140005354BB40491C18440329E4DBE9E7F0B5DC
:1011500005460020044602462C4B4FF4007700E081
:10116000641C2E5D36B102EB040C9C449CF800C458
:10117000B445F5D0032C3ED302F580601844047FBB
:10118000457FC67F04EB0524857F2D0405EB0665AE
:101190002C4451EA04052AD021B919494968403143
:1011A0008C4224D8174C00216C3455181D4495F8F6
:1011B00000546554491C0C29F7D3817EC27E01EB93
:1011C0000221027D407D120402EB00600C182046D3
:1011D000FFF797FF40F6F57502E000BFFFF791FFBC
:1011E000C11EA942FAD3A0F57061FF3901D00020D9
:1011F000F0BD2046F0BD2032BA42B2D3F0BD0000AF
:10120000DC0000100808001055534243C8010010CC
:10121000FFB558A60446E1CE8DE8E100022902DAC6
:10122000002004B0F0BD6018002100F8011D6946DF
:10123000B3FBF2F502FB1535B3FBF2F34D5D00F89D
:10124000015DA042F4D8ECE7024600203F2A06D117
:101250004A78342A03D18978322900D10120704795
:1012600002004FF0000009D0012A0ED0022A04D15A
:10127000C978662907D0462905D07047C9786529FD
:1012800001D04529F9D101207047C9786E29FAD0DB
:101290004E29F8D07047F0B50646002004460546B2
:1012A0000346F25CA2F13007092F01D8FDB209E034
:1012B000A2F14107052F02D8373AD5B202E0613AD0
:1012C000052A05D95B1CDBB205EB0414042BE8D31B
:1012D0000988A14200D10120F0BD10B501F045FA06
:1012E0002848294C006840B101F0ADFBA0F5F4207E
:1012F000206001F0A8FB606010BD01F0A4FB6FF45A
:1013000074210844206001F09EFB6FF4F42108442E
:10131000F1E7F8B51C4D034600242E687018696883
:1013200087188F4200D9881A00920246304601F091
:10133000A7FA2046F8BD0B460146134810B50068D1
:101340000024184401F0C8FC204610BD70B50022EE
:101350000D4C134608340AE0E65C855C5B1C754066
:10136000DBB28554402B00D30023521CD2B28A42F8
:10137000F2D370BD303132333435363738394142EB
:1013800043444546CC0000101401001030B4554CC5
:10139000534A0323C4F8B031136843F48033136015
:1013A000514A30BC104710B572B633244F4B10C3AE
:1013B00007C34F484FF47A710068B0FBF1F0186032
:1013C000191D4A48FFF7E2FF62B610BD474A3223B3
:1013D0001360C2E9010146484FF47A710068B0FB1E
:1013E000F1F0D06002F114011046CFE73F4A3423F8
:1013F0001360C2E901013E484FF47A710068B0FB06
:10140000F1F0D06002F114011046BFE710B572B6DA
:101410000624384951F82420824212D935497839B6
:1014200051F82410814207D121460846FFF7CEFF2C
:1014300021460846FFF7DAFF21460846FFF7C6FFB8
:1014400002E0641C1D2CE5D962B610BD2DE9F04107
:10145000294C236803B92060244D00202835636897
:1014600003E00F5C1E18401CAF559042F9D398184A
:101470004FF480766060B04213D12068FFF7C6FF5A
:101480001A4D1435286800B1FEE718493246283154
:101490002068FFF788FF286800B1FEE70020606041
:1014A00020600020BDE8F08114494FF4C04008607E
:1014B000FEF722BE46F2044000210088A0F5194242
:1014C000993A0AD04FF4C0404FF4002208C8904225
:1014D0001944FBD309B10020704701207047000078
:1014E00088C10F4000C00F40F11FFF1F800800108F
:1014F00074010010D83200005C01001008ED00E01B
:10150000002070475849C20702D04FF000728A6726
:10151000800702D54FF080608867002070475249ED
:10152000C20702D04FF00072CA67800702D54FF0A1
:101530008060C86700207047014600204A4ACB07F8
:1015400003D0536F9B0100D50120890704D5516F4B
:10155000490101D540F00200704710B50446FFF77D
:10156000EBFF0346FFF7DBFF24EA0300FFF7CAFFA8
:10157000002010BD10B53D4B38B159680424042932
:1015800006D2DFE801F0061D37540020586098604D
:1015900010BD042807D005280AD0012402285ED0F7
:1015A00001284CD010BD0320FFF7B9FF01201EE039
:1015B000BDE810400120B2E7FFF7A4FF5C6010BD5A
:1015C000062808D00328FAD00928ECD00D280AD024
:1015D0000C28E8D010BD0320FFF7A1FF0220FFF781
:1015E00091FF022021E00320FFF799FF0220BDE8D0
:1015F000104087E7062808D00A280FD009281ED0F7
:101600000C28D0D00D28EED010BD986810F01F0F18
:1016100000F101009860F7D102201DE00320FFF7E0
:101620007EFF0120FFF76EFF0320586010BD0728E2
:101630000AD00A28B7D00B2811D00928F6D10320E8
:10164000FFF76DFF0120B7E7986810F01F0F00F15A
:1016500001009860EAD10120BDE810407DE7032039
:10166000FFF75DFF0220A7E7008009206801001056
:10167000F0B57248D0F804114FF00002CB05704964
:1016800028D4D0F80C31DC076E4B03D0D0F8A04141
:10169000640660D5D0F80441E40605D0D0F80441D2
:1016A00004F01F04B3FBF4F40C60D0F8A851ED066D
:1016B0000ED0D0F8A85105F01F05B3FBF5F34B6031
:1016C000D0F8003103F001035B1CB4FBF3F331E00D
:1016D0000023F4E7D0F88830DB053CD5D0F80C3196
:1016E000DB0703D0D0F8A0315B0634D5D0F88830C2
:1016F000D0F8044103F01F0314F01F05D0F8A841EF
:10170000D0F8006104F01F0406F0010603F10103A4
:1017100006F1010603D04B4F5F43B7FBF5F50D60B3
:1017200024B1484F7B43B3FBF4F300E000234B604C
:10173000B5FBF6F3C1F80830D0F80831DB05D0F876
:1017400008311CD513F01F0303D0042B07D0062B40
:1017500005D0CA60F0BD0A604A608A60ECE7D0F844
:101760008820D0F8083102F01F02D0F80C0103F0F5
:101770001F033448521C4243B2FBF3F00FE09B05B9
:10178000E7D5D0F80C21D20702D0D0F8A80001E0AC
:10179000D0F888002B4A00F01F00401C5043C8605E
:1017A000F0BD264810B42021C0F8A011D0F8A01137
:1017B0004906FBD50121C0F80C110922C0F884208C
:1017C000C0F88010AA22C0F88C205523C0F88C30B5
:1017D000D0F888406405FBD52324C0F8A440C0F8A5
:1017E000A010C0F8AC20C0F8AC3000BFD0F8A820E2
:1017F0005205FBD540F20112C0F8042140F201224B
:10180000C0F80821C0F800110221C0F8B411042169
:10181000C0F8A8110C49C0F8C4100021C0F8C811C4
:10182000D0F8B02142F00302C0F8B02145F23A02EC
:1018300002600648016010BC1AE7000000C00F40BB
:1018400074010010001BB700FE9FF8F708ED00E0E0
:10185000F0B5AE49032008630020C1F80801AC4888
:1018600004228265026C42F004020264A94A8A667C
:1018700000220A611022C261026822F01002026096
:101880000322C1F87022C1F8742200224A644FF486
:1018900000328261026842F4003202600922C1F81B
:1018A0000021C1F804211022C1F8D420520482631F
:1018B000026A42F4001202620D22C1F8D020C1F87F
:1018C000E0200022C1F8F4204FF00052C263026A07
:1018D00042F0005202620022C1F8F0204FF0805224
:1018E000C263026A42F0805202621022CA67020496
:1018F0008261026842F0004202601022C1F81421A5
:1019000020278765026C42F0200202641022C1F891
:101910001C218022C265026C22F0800202649026A3
:10192000C1F8FC600204C263026A22F00042026253
:101930001022C1F8DC20D204C263026A22F4000241
:10194000026201220A66CA654A660323C1F8D830DA
:101950000523C1F8E4308A601123CB60CA630B64AD
:101960000224C1F820411225C1F824510C604D60B9
:101970000C604D6010248C659405C461046844F4C7
:10198000800404600124CC630B641023C1F82C3163
:10199000CB14C365036C43F4006303641023C1F8E4
:1019A00030318B14C365036C43F48053036440F2FD
:1019B00082234B629A240C62CB6110234B618761B6
:1019C000036843F02003036010238B61402484618B
:1019D000036843F04003036001230B67CB6640F2CA
:1019E0000243CB628B621023C1F8E8309306836315
:1019F000056A45F0806505621025C1F8EC50D506F2
:101A0000C563056A25F0006505624E635503C5612F
:101A1000056825F4005505600025C1F8E851C36745
:101A2000036E43F080630366C1F8E4515306C36755
:101A3000036E43F0007303668A23C1F8F83008236D
:101A4000C1F8C8309504C563066A46F4802606626C
:101A50001026C1F828610E15C665066C26F480664E
:101A600006640126C1F88060C1F88460C1F8906006
:101A7000C1F8A060C1F8A460C1F8A860C1F8B8605E
:101A8000C1F8BC60C1F8C060C1F8C4600026C1F8EC
:101A90001861C465046C44F0400404640B651405CB
:101AA000C461046824F480140460CB64D404C46169
:101AB000046824F4002404608B64C561046824F481
:101AC000802404600024C1F80C418365036C43F05A
:101AD00008030364C1F8104110238365036C43F0CD
:101AE000100303640C480D4B0068984204D141F880
:101AF000B82F8A60CA60F0BD094A9042FBD18120AC
:101B000041F8B80F8860C860F0BD000000C0024016
:101B1000008009200200010064010010473F1927DE
:101B2000473F19474D4900200867C86002224A61B3
:101B300088613022CA634A498A684A49C1E900205B
:101B400049490860494908607846494908600020C9
:101B500070472DE9F04341F288320024424F434E52
:101B6000434B904208D8642800D228B942F2107240
:101B7000914201D8052907D2862038607846346022
:101B800018608620BDE8F083DFF8D490D9F80850BB
:101B9000344AD2F800C0A5EB0C05D2F804C00CEB17
:101BA0004C08C8EBCC1CB5EBCC0F06D20520386036
:101BB0007846346018600520E4E7284D4FF0020CA9
:101BC000C5F804C048B1DFF8AC80B8FBF0F04010B5
:101BD000A861C5F804C001206860D9F80800C2E90E
:101BE00000013C607846346018600020CAE770B598
:101BF0001C4C00250E466560FFF7ABFF1A49000636
:101C000001D5086870BD164B06EB46022068C2EB92
:101C1000C6129E68361AB6EBC20FFAD30F480222DC
:101C20004260C26B02F0FE02C2636560E9E70C48E5
:101C300080680C490A68801A4A6802EB4203C3EBC9
:101C4000C212B0EBC20F08D3044802224260C26B3A
:101C500002F0FE02C263002048607047008000402E
:101C60000000094088010010D0000010D4000010CE
:101C7000D800001080C3C901FA4800214FF00112BA
:101C8000818001704170C0E902217047F5491C3123
:101C9000002000F0A3BB10B5F24C1434A288402AF7
:101CA00000D940228020216800F0C9FB216801444E
:101CB0002160A188081AA08010BD10B5E94C002051
:101CC0001434216800F08AFB216801442160A18856
:101CD000081AA08010BD00221146802000F0AFBB82
:101CE000E149002000F07ABB70B5DE48DD4D1C30C4
:101CF00005F11405007810F01F040AD0D949DA4B19
:101D000001F11C004A780079012C06D0022C26D162
:101D100009E0D448001D28601DE002B3897888429C
:101D20001DD2002015E000F08F04200605D504F038
:101D30000F064FF48030B04001E00120A0400AB906
:101D400022070CD18A68024209D0C9680142E8D052
:101D5000012018802B60FFF79EFF012070BD00203E
:101D600070BD024670B5BF48BE4C1C30017811F002
:101D70001F030146498804D0012B29D0022B27D10B
:101D800011E0012924D132B1012000F0C2FAA0886B
:101D900040F0020005E0002000F0BBFAA08820F02F
:101DA0000200A08021E0007900F08F00030605D535
:101DB00000F00F034FF480359D4001E00125854080
:101DC00063782BB1030703D0A3682B4200D009B17D
:101DD000002070BD22B100F0EDFAE068284303E076
:101DE00000F0F2FAE068A843E060012070BD9D4871
:101DF00010B51C30007810F01F0F9A4800F11C003D
:101E0000C0782AD197491431012807D001F108027E
:101E10000228937806D003281FD112E09348086067
:101E2000122012E09248002204E004780CB14488A9
:101E30002044521C9342F8D1027872B10860408865
:101E400003E08C481844086000788A88824200D9F0
:101E50008880FFF720FF012010BD002010BD2DE974
:101E6000F84F804F00201C370090B8787D4E4FF01F
:101E700000094FF0010A4FF4803B00286BD07C4CE6
:101E800065E06078022804D0042841D005285CD1A0
:101E900041E06179B878814238D170702079B070B2
:101EA0007049002011F1100101F80090401C042835
:101EB000FAD301254FEA06080AFA05F0D8F8081007
:101EC000084202D0284600F061FAD8F808100BFA50
:101ED00005F0084203D045F0800000F057FA6D1C71
:101EE000102DE9D34FF00110C8E90209012000F0DC
:101EF00011FAE0794006B8F8040002D540F001007C
:101F000001E020F00100A8F804001EE060881DE058
:101F1000E078009019E00098B8B9A07800F08F053B
:101F2000280604D505F00F010BFA01F001E00AFACA
:101F300005F0B16801432046B16000F000FA284680
:101F400000F01AFA284600F02BFA20780444207892
:101F5000002896D11FE086F8019001245546D84606
:101F6000B16805FA04F0084202D0204600F00EFAEB
:101F7000B16808FA04F0084203D044F0800000F091
:101F800005FA641C102CEBD34FF00110C6E90209CE
:101F9000002000F0BFF9B8787178884202D10120A2
:101FA000BDE8F88F0020FBE72DE9FC5F2D4D0027F1
:101FB0003E466878BB46B846002871D0BA462C4CDD
:101FC00005F11C0968E06078022804D0042808D0D4
:101FD00005285FD119E06079697888425AD0608815
:101FE00059E0A77899F80410E6784FF00008B94254
:101FF00050D199F80200B0424CD11A484FF0010A72
:10200000103010F807B0C65544E099F80410B942F2
:1020100040D1A17801F08F010191090605D5019900
:1020200001F00F024FF4803101E0019A012191404B
:10203000009199F80200B0421ED1A8680843A86038
:10204000E968009881432046E96000F078F901983A
:1020500000F092F9019800F0A3F9009948EA01080C
:1020600018E0000090010010A8090010EA0200002A
:1020700050330000713300005E450BD118EA010FA8
:1020800008D1A8688843A860E8688843E860019898
:1020900000F07CF9207804442078002893D1504641
:1020A000BDE8FC9F2DE9F041494C0027A4F108064A
:1020B0002178A4F11C05082863D2DFE800F062044F
:1020C000647262628381FFF7E1FD2078C00900F04D
:1020D00052F9E088B0802078C0F34111F1BB6178FB
:1020E0000C294AD2DFE801F00609490B49101A1DF4
:1020F0001F253142FFF7F8FD4DE0002000E00120F0
:10210000FFF72FFE50B306E010F01F0F35D1A07877
:1021100040F080002870BDE8F041DCE5FFF767FE85
:1021200039E000202AE010F01F0F26D128481B3884
:102130001AE010F01F0F20D1FFF791FE70B1FFF7EA
:10214000CAFDBDE8F041FEF7A3B800F01F0001286A
:1021500013D1687810B12079A97800E00DE08842A9
:102160000BD21B490C39084430601CE000F01F0002
:10217000012802D1FFF718FFC4E7802000F01AF908
:10218000B780BDE8F081080608D4B0880028F8D0F0
:10219000FFF793FDB0880028EFD0F2E7BDE8F041EB
:1021A0009EE5080602D5BDE8F04174E528780106F1
:1021B000E7D500F07F002870BDE8F04100F054B88A
:1021C000802000E00020BDE8F04100F0FDB80000F4
:1021D000AC01001001460007C00E090600D5401CE6
:1021E0007047DC491022C1F80822C1F8100200BF74
:1021F000D1F80002C006FBD57047D64A1023C2F8BA
:102200000832C2F8100200BFD2F80002C006FBD5A7
:10221000C2F80832C2F81012D2F80002C006FBD58C
:102220007047CC493022C1F80822C1F8100200BF23
:10223000D1F800028006FBD5D1F81402704710B522
:10224000040001D0012000E000204FF4807141EA39
:102250000041C148FFF7D1FFC0494FF480200CB1C5
:10226000886310BDC86310BD30B5BD49BD4D41EA9E
:10227000004421462846FFF7C0FF21462846BDE816
:102280003040BAE7B3480021C0F848124021C0F8F6
:102290004C120122C0F84822C0F84C12D0F80012AB
:1022A000C905FBD54FF0FF31C0F83812C0F8341221
:1022B000C0F808120C21C0F80412704730B5AA4CBF
:1022C0001A202060221D116830EA0101FBD1A749C4
:1022D00001234B678B679F4D0023C5F810318A237C
:1022E000C1F8F8302060116830EA0101FBD14FF0ED
:1022F000E0214FF08070C1F880029D4B202283F8CE
:102300000024C1F80001FFF7BDFFBDE83040002008
:10231000AAE7704710B500B101204FF4807444EA79
:1023200000419448FFF769FF8A480321C0F844122E
:10233000D0F80012C905FBD5C0F8084210BD10B591
:1023400002468078FFF746FF8249D1F844320124E3
:1023500084402343C1F84432C1F848029088C1F850
:102360004C0200BFD1F80002C005FBD54FF48070CD
:10237000C1F8080210BD704700B5FFF72BFF7E497A
:102380005DF804EB41EA0040891336E700B5FFF73A
:1023900021FF79495DF804EB41EA004077492CE7D9
:1023A00000B5FFF717FF74495DF804EB41EA004000
:1023B000891322E700B5FFF70DFF6F495DF804EBC5
:1023C00041EA00406E4918E700B5FFF703FF6A498C
:1023D0005DF804EB41EA004089130EE700F00F02BC
:1023E000012370B503EB82035A4AC2F8283200BFBA
:1023F000D2F820321C05FBD5C3F309030024DD1CF1
:1024000005E000BFD2F8186241F8046B641CB4EB1D
:10241000950FF7D30021C2F8281241F24821C1409C
:10242000C9070AD1FFF7D6FE4FF4A06141EA004088
:10243000FFF7D7FE5348FFF7D4FE184670BD70B5BE
:1024400013460546434C00F00F00022202EB8000C9
:10245000C4F82802C4F824320020DA1C05E000BFCA
:1024600051F8046BC4F81C62401CB0EB920FF7D318
:102470000020C4F828022846FFF7ACFE4FF4A06104
:1024800041EA0040FFF7ADFE3F48FFF7AAFE1846BD
:1024900070BD2DE9F0412F4DD5F80032C5F8083256
:1024A000180721D52C48FFF79CFE3848FFF7B9FEE6
:1024B000C10605D5FFF7E6FEBDE8F041FDF7D9BE40
:1024C000810705D5BDE8F04100F00100FDF7CBBE66
:1024D000010709D5400703D5BDE8F041FDF7D0BE9F
:1024E000BDE8F041FDF7D3BE294E58074FF0010774
:1024F0001CD4BDE8F0810024D5F8302207FA04F19D
:102500000A4210D06008C5F8381200BFD5F8001292
:102510008906FBD5D5F81412E2070CD056F8201026
:1025200009B103208847641C202CE5D3D5F830027C
:102530000028E0D1DDE73CB9490705D5316819B17C
:10254000012088470124D7E756F820100029EAD057
:102550000220E7E700C008200005FE0000800920F7
:10256000000180000005D000F4CF082000C0024028
:1025700018E000E00005D800000540000001200040
:10258000000101000005F2000005FA000002FE0053
:10259000E43300002DE9F047FE4E80464FF080778F
:1025A00030684024FC4DB84249D100BF00BF00BF95
:1025B00000BF00BF00BF00BF00BF00BF00BF00BF23
:1025C00000BF00BF00BF00BF00BF00BF00BF00BF13
:1025D00000BF00BF00BF00BF00BF00BF00BF00BF03
:1025E00000BF00BF00BF00BF00BFEC611520FDF7BA
:1025F0009BFE0020FDF798FE00F0FF09AC6100BFD4
:1026000000BF00BF00BF00BF00BF00BF00BF00BFD2
:1026100000BF00BF00BF00BF00BF00BF00BF00BFC2
:1026200000BF00BF00BF00BF00BF00BF00BF00BFB2
:1026300000BF00BF00BF00BF00BF00BF00BF00BFA2
:1026400000BF00BF00BF00BF00BF00BF00BF00BF92
:1026500000BF00BF00BF00BF00BF00BF00BF00BF82
:1026600000BF00BF00BF00BF00BF00BF00BF00BF72
:1026700000BF00BF00BF00BF00BF00BF00BFEC61D4
:102680000620FDF751FEAC6100BF00BF00BF00BFD8
:1026900000BF00BF00BF00BF00BF00BF00BF00BF42
:1026A00000BF00BF00BF00BF00BF00BF00BF00BF32
:1026B00000BF00BF00BF00BF00BF00BF00BF00BF22
:1026C00000BF00BF00BF00BF00BF00BF00BF00BF12
:1026D00000BF00BF00BF00BF00BF00BF00BF00BF02
:1026E00000BF00BF00BF00BF00BF00BF00BF00BFF2
:1026F00000BF00BF00BF00BF00BF00BF00BF00BFE2
:1027000000BF00BF00BF00BFEC610120FDF70CFE61
:102710004FEA8800FDF708FE3068B84202D148460B
:10272000FDF702FEAC6100BF00BF00BF00BF00BFED
:1027300000BF00BF00BF00BF00BF00BF00BF00BFA1
:1027400000BF00BF00BF00BF00BF00BF00BF00BF91
:1027500000BF00BF00BF00BF00BF00BF00BF00BF81
:1027600000BF00BF00BFBDE8F0872DE9F0474FF084
:10277000000900BF00BF00BF00BF00BF00BF00BF17
:1027800000BF00BF00BF00BF00BF00BF00BF00BF51
:1027900000BF00BF00BF00BF00BF00BF00BF00BF41
:1027A00000BF00BF00BF00BF00BF00BF00BF00BF31
:1027B00000BF4025784EF5619F20FDF7B5FD002054
:1027C000FDF7B2FD00F0FF080020FDF7ADFDC4B23B
:1027D0000020FDF7A9FDC1B2B56100BF00BF00BF79
:1027E00000BF00BF00BF00BF00BF00BF00BF00BFF1
:1027F00000BF00BF00BF00BF00BF00BF00BF00BFE1
:1028000000BF00BF00BF00BF00BF00BF00BF00BFD0
:1028100000BF00BF00BF00BF00BF604D604E614FF2
:10282000B8F1C20F01D1202C07D0822028602120CE
:10283000306078463860822095E75648142912D0D7
:10284000152913D0162915D0182916D0C0F80090D4
:102850000020FFF79FFEC5F800907846C6F800906C
:10286000386000207FE74FF4801101E04FF4001141
:102870000160EDE74FF48001FAE74FF08071F7E770
:102880002DE9FF4F8DB00D46DDF868900026434CD2
:1028900007935FEA09013ED04FF4805701463A465C
:1028A0006846FDF797FCDDE900B10C913A46691CDA
:1028B0006846FDF78FFCDDE90010CDE904013A46DA
:1028C00068460F99FDF786FCDDE90085A9EB060750
:1028D000C5F58050B84200D2074625B1D8457DD114
:1028E0000C9885427AD14FF4805000F04BFC5FEA9F
:1028F000000A1CD0D8455BD10C98854258D12A4695
:102900004FEA0830514600F0F0F8000619D550465D
:1029100000F010FC85E0862020602148092101603C
:10292000784620490860862011B0BDE8F08F8220EB
:1029300020601B482221016079461A4801608220EC
:10294000F2E70598804509D1049901EB0030C1F503
:102950008052514400F0C9F80006D8D4404600F037
:1029600041F90006D3D407983A46811905EB0A00CD
:10297000FDF7A2FCEA194FEA0830514600F018FBB7
:102980000006C4D4059988453ED1049800EB013077
:10299000049909E0BC01001000800920D00000105B
:1029A000D4000010D8000010C1F58052514427E037
:1029B000059988450AD1049800EB01300499C1F5C6
:1029C0008052514600F091F80006A0D4404600F035
:1029D00009F900069BD40798811900E018E00F98C8
:1029E0003A46304400F0E4FA000690D40599884550
:1029F0000AD1049800EB01300499C1F58052514688
:102A000000F0D6FA000682D4504600F093FB0AE0AC
:102A100007983A4681190F98304400F0C9FA000629
:102A200001D5206880E73E44002508F101084E45A5
:102A3000FFF44CAF05490020206008607846044947
:102A40000860002070E7034800687047D400001059
:102A5000D8000010BC01001070B500BF00BF00BF5F
:102A600000BF00BF00BF00BF00BF00BF00BF00BF6E
:102A700000BF00BF00BF00BF00BF00BF00BF00BF5E
:102A800000BF00BF00BF00BF00BF00BF00BF00BF4E
:102A900000BF00BF00BF00BF00BF4025CE4CE561B6
:102AA0000620FDF741FCA56100BF00BF00BF00BFCD
:102AB00000BF00BF00BF00BF00BF00BF00BF00BF1E
:102AC00000BF00BF00BF00BF00BF00BF00BF00BF0E
:102AD00000BF00BF00BF00BF00BF00BF00BF00BFFE
:102AE00000BF00BF00BF00BF70BD2DE9FC5FBB4D44
:102AF000BB4EBC4F5FEA020A8B4604464FF000080B
:102B00000DD001A9B84800F001F980B182202860F9
:102B100021203060784638608220BDE8FC9FC5F8EF
:102B200000807846C6F8008038600020F5E7032072
:102B30008DF80000200C8DF80100200A8DF80200AD
:102B40008DF8034000BF00BF00BF00BF00BF00BF43
:102B500000BF00BF00BF00BF00BF00BF00BF00BF7D
:102B600000BF00BF00BF00BF00BF00BF00BF00BF6D
:102B700000BF00BF00BF00BF00BF00BF00BF00BF5D
:102B800000BF00BF944C4FF04009C4F81C900421D2
:102B90006846FDF7D0FB51465846FDF7D8FBC4F810
:102BA000189000BF00BF00BF00BF00BF00BF00BF44
:102BB00000BF00BF00BF00BF00BF00BF00BF00BF1D
:102BC00000BF00BF00BF00BF00BF00BF00BF00BF0D
:102BD00000BF00BF00BF00BF00BF00BF00BF00BFFD
:102BE00000BF9CE72DE9FC47044601A97E4800F0A0
:102BF0008DF87A4D7A4EDFF8EC9148B1822028604A
:102C00002220794630608220C9F80010BDE8FC8798
:102C10009DF80400800701D4FFF71EFF20208DF8E7
:102C2000000020098DF8010020018DF80200002429
:102C30008DF8034000BF00BF00BF00BF00BF00BF52
:102C400000BF00BF00BF00BF00BF00BF00BF00BF8C
:102C500000BF00BF00BF00BF00BF00BF00BF00BF7C
:102C600000BF00BF00BF00BF00BF00BF00BF00BF6C
:102C700000BF00BF4027DFF86081C8F81C70042146
:102C80006846FDF758FBC8F8187000BF00BF00BFCA
:102C900000BF00BF00BF00BF00BF00BF00BF00BF3C
:102CA00000BF00BF00BF00BF00BF00BF00BF00BF2C
:102CB00000BF00BF00BF00BF00BF00BF00BF00BF1C
:102CC00000BF00BF00BF00BF00BF2C60794634606A
:102CD0000020C9F8001099E770B5414D414E3F4CB6
:102CE0002AB1FFF702FF000609D5206870BD8620D3
:102CF00020600920286078463060862070BD002062
:102D00002060286078463060002070BD2DE9F041D9
:102D1000364C0F460646A56806E0A068401BB04248
:102D200002D30120BDE8F081384600F003F8002806
:102D3000F3D1F7E770B5044600BF00BF00BF00BF86
:102D400000BF00BF00BF00BF00BF00BF00BF00BF8B
:102D500000BF00BF00BF00BF00BF00BF00BF00BF7B
:102D600000BF00BF00BF00BF00BF00BF00BF00BF6B
:102D700000BF00BF00BF00BF4025174EF561052012
:102D8000FDF7D2FA0020FDF7CFFA2070B56100BF41
:102D900000BF00BF00BF00BF00BF00BF00BF00BF3B
:102DA00000BF00BF00BF00BF00BF00BF00BF00BF2B
:102DB00000BF00BF00BF00BF00BF00BF00BF00BF1B
:102DC00000BF00BF00BF00BF00BF00BF00BF207832
:102DD00000F0010070BD000000800920D00000104C
:102DE000D4000010D8000010A086010000000940A7
:102DF0002DE9F34F85B0044603A9B24800F0FDF871
:102E0000B14DB24EB24F4FF0820B18B12120C5F830
:102E100000B060E0FFF720FE42208DF800004FF088
:102E2000000ACDF801A0CDF805A0ADF809A000BFBB
:102E300000BF00BF00BF00BF00BF00BF00BF00BF9A
:102E400000BF00BF00BF00BF00BF00BF00BF00BF8A
:102E500000BF00BF00BF00BF00BF00BF00BF00BF7A
:102E600000BF00BF00BF00BF00BF00BF00BFDFF852
:102E700064924FF04008C9F81C800B216846FDF7AA
:102E80005AFAC9F8188000BF00BF00BF00BF00BFDA
:102E900000BF00BF00BF00BF00BF00BF00BF00BF3A
:102EA00000BF00BF00BF00BF00BF00BF00BF00BF2A
:102EB00000BF00BF00BF00BF00BF00BF00BF00BF1A
:102EC00000BF00BF00BF03A97E4800F096F848B1DC
:102ED0002220C5F800B0306078463860822007B004
:102EE000BDE8F08F9DF80C00800701D4FFF7B4FD1A
:102EF00002208DF80000200C8DF80100200A8DF8CA
:102F0000020006988DF803408DF8040000BF00BF52
:102F100000BF00BF00BF00BF00BF00BF00BF00BFB9
:102F200000BF00BF00BF00BF00BF00BF00BF00BFA9
:102F300000BF00BF00BF00BF00BF00BF00BF00BF99
:102F400000BF00BF00BF00BF00BF00BF4446C8466F
:102F5000C9F81C4005216846FDF7EDF9C8F818408E
:102F600000BF00BF00BF00BF00BF00BF00BF00BF69
:102F700000BF00BF00BF00BF00BF00BF00BF00BF59
:102F800000BF00BF00BF00BF00BF00BF00BF00BF49
:102F900000BF00BF00BF00BF00BF00BF00BF00BF39
:102FA000C5F800A07846C6F800A03860002096E773
:102FB0002DE9F05F444EDFF81491DFF814A11500FD
:102FC00083460F464FF000080ED000240AE0395D1A
:102FD0000BEB0400FFF70CFF000602D53068BDE8DC
:102FE000F09F641CAC42F2D3C6F800807946C9F861
:102FF00000800020CAF80010F1E72DE9F041364CBE
:103000000F460646A56806E0A068401BB04202D302
:103010000120BDE8F081384600F003F80028F3D124
:10302000F7E770B5044600BF00BF00BF00BF00BF98
:1030300000BF00BF00BF00BF00BF00BF00BF00BF98
:1030400000BF00BF00BF00BF00BF00BF00BF00BF88
:1030500000BF00BF00BF00BF00BF00BF00BF00BF78
:1030600000BF00BF00BF40251A4EF5610520FDF7E7
:103070005BF90020FDF758F92070B56100BF00BF73
:1030800000BF00BF00BF00BF00BF00BF00BF00BF48
:1030900000BF00BF00BF00BF00BF00BF00BF00BF38
:1030A00000BF00BF00BF00BF00BF00BF00BF00BF28
:1030B00000BF00BF00BF00BF00BF00BF207800F00E
:1030C000010070BDA0860100D0000010D4000010E7
:1030D000D8000010008009200000094070B58C184D
:1030E00010F8015B15F0070301D110F8013B2A111C
:1030F00006D110F8012B03E010F8016B01F8016B09
:103100005B1EF9D12B0705D40023521E0DD401F804
:10311000013BFAE710F8013BCB1A921C03E013F8CD
:10312000015B01F8015B521EF9D5A142D8D3002002
:1031300070BD000010B5002821D0114B0022001FE7
:10314000196803E0814203D80A4649680029F9D189
:1031500052B11368841A9C4204D10068184410606C
:10316000104602E0506000E0186039B102680B1AA6
:10317000934203D10B681A4402604968416010BD54
:10318000C0010010F0B50B30154D20F007010024F0
:10319000144A0FE003688B420BD38B4205D95E1AA9
:1031A00043184768C3E9006700E04368136002C042
:1031B00004E0021D10680028ECD12046002802D14E
:1031C000286808B10020F0BD064A07481060074A89
:1031D000121A22F00702C0E9002401202860D7E774
:1031E000C4010010C0010010EC090010E8790010C3
:1031F000EB3C904D53444F53352E300002020100FA
:103200000110000004F802000100010000000000AD
:1032100000000000000029EFBEADDE41544F4C20FD
:10322000465072696E7446415431322020200000AD
:1032300034340000243400004034000044340000E2
:103240005034000038340000303400002C340000CA
:103250003C340000483400004C34000028340000A6
:1032600000000000001000000020000000300000FE
:1032700000400000005000000060000000700000EE
:10328000008000000090000000A0000000B00000DE
:1032900000C0000000D0000000E0000000F00000CE
:1032A0000000010000800100000002000080020018
:1032B0000000030000800300000004000080040000
:1032C00000000500008005000000060000800600E8
:1032D0000000070000800700FF0F0000FF1F000034
:1032E000FF2F0000FF3F0000FF4F0000FF5F0000C6
:1032F000FF6F0000FF7F0000FF8F0000FF9F0000B6
:10330000FFAF0000FFBF0000FFCF0000FFDF0000A5
:10331000FFEF0000FFFF0000FF7F0100FFFF010043
:10332000FF7F0200FFFF0200FF7F0300FFFF03009B
:10333000FF7F0400FFFF0400FF7F0500FFFF050083
:10334000FF7F0600FFFF0600FF7F0700FFFF07006B
:103350000902200001010080320904000002080671
:10336000506207058202400000070502024000008B
:1033700000040309041C03410054004F004C0020CA
:10338000002000200020002000200020002000203D
:1033900000280346005000720069006E007400208F
:1033A0000046006C006100730068002000200020CF
:1033B0000020002000200020001A0346006900724F
:1033C000006D007700610072006500300030003051
:1033D0000030000E034D0065006D006F0072007933
:1033E00000000000A5200000000000009302000083
:1033F00000000000000000000000000000000000CD
:1034000000000000000000000000000000000000BC
:1034100000000000000000000000000000000000AC
:103420000000000046656200446563004175670066
:103430004A756C004A616E004A756E0053657000F3
:103440004D617200417072004F6374004E6F7600E0
:103450004D617900A00D41544F4C20465072696E69
:1034600074280546D4284B3D39609F4574616C6FC4
:103470006E609920126612341232124E1230120F00
:103480001BDE30071230122E12663272326D1E466B
:1034900034324E30011546524D202008BC4197373A
:1034A000383738263D6E2B380243A0071B106004C6
:1034B000411AFF01014C100D455F5553494E475FBE
:1034C0004D4F5645B81328085838365F54554E4569
:1034D0005F4550494C4F47551F8A291F175348498C
:1034E00046543103192A0810080E270780C3C90162
:1034F000148793031B6CDCC9014200002619BB9E94
:1035000006FE8689E4D58ABA1D167E5AA0E29591F8
:10351000A57DFF39B430A385E65AFD21E534B445D5
:103520008DF75FC1AE949676B96F4CFC2CD878803D
:103530001232FC6ABC8FE17336D00D23C8794C9DE2
:103540002DB93F02B8E2218D85BACFE663BB8CD19D
:10355000E958DFED9F153844EFD57F1BA1C24D6EB2
:10356000832DE67E910ADB6266C1D1467D0C88F22E
:10357000BFA0129BB92FC73D02C14E14F0B0543703
:103580001BE02A34272A4DCDB7F681CEE814C8E0D7
:1035900042015952395AC005F2EEB735ECAB80EE14
:1035A000AD416C42F2D142F0EE0DA64B929DDEC4CD
:1035B000294586A84689639DBDA9ECCE61CE5812E7
:1035C000B929D7DBA3BB004F4898EEE7C5A3BF00DE
:1035D0006CA0EFB75E7797D0FEC06D378DF6F5C55E
:1035E0002C1284719D135510622196C8A8BB5ACF26
:1035F00072602E04F4DBB178087FAA3551B1C70E92
:10360000478B59A597E223087E8F03575891182EB0
:103610002CB31875B6A94EE3766873CAD1AEA8D894
:1036200052B4A8BD69E9759B613A172EC03CE11DF3
:103630009F5169F097B5E44621704A1C38EDC40BE0
:1036400095EBB586B00152E3846048E92C6095C2E1
:103650004878863D551EBA3E45986280BB3C099B22
:10366000CC2EBDAF82988CE77949956EA4379B1616
:10367000F00B4150900F38B4F2FD827B10D136AE82
:1036800076B95BC3CEAD8B6BBD47334A2ECEE27DA0
:10369000F31231DDFA529DF1BB7FCE5F8FCA9AAE35
:1036A000A82FC9F7B24439EC81C151F2C319FAA469
:1036B00007764DA9623EFAE21A95B412415D326B6B
:1036C000B25235A8536A33DA57DD12A3DF3BBE810D
:1036D0007739BAB00FD4556C324102CAD4FA81E1BD
:1036E000AEB95C9B5CB125B5E5776CEF2C81FB77BF
:1036F000BC96CB39771D2567822C5309A42E73AE57
:10370000DB185E9865730EC73123F545C0976F616E
:103710006A1C8FACA08468D5B015538616C5E21C10
:10372000DD91B9335903D9B2C87E727907DF2C1500
:103730004AAAE3CC06424DD9754E580952AECF0382
:10374000340B82E795C1AC30A2EB72AA64A4F3E615
:1037500078E4463EAD489B71B196D4B90A20FD226B
:1037600025F0D691B28FD261A1D7F3BE0CAFF60A85
:10377000BACDEAFB93A117937A12BB117BD2C8BFD3
:10378000C4FB7C71C557367C00026FBE02AF97E068
:10379000DABD3181C0E3E4CC9187C027224E827A22
:1037A000261B00711597485869752C72C17ECF6A27
:1037B0003B693A89FAFDC2C7F1CE3ABFDA55C63342
:1037C000B7C966D9CE5E4BB6AB25BE98EB0F310CB0
:1037D0002C7DE2555E92451F21F3059F56CB06BC1A
:1037E0007827D440B650704B0A6D398E94796DA10C
:1037F0005E0C6B76EF9701374678F2F527B987971D
:1038000035B697AF6774067920C931056C28A328AF
:10381000D8000B9B273262D01E7E9561C036DAC07D
:103820005F823B9216E153DE1F4A5940222D57CB4F
:103830001CC0CE0E4D4FF5C896D0F4052CF68276FE
:103840006A313292B36BCCB7D62967575ABAB725CB
:103850004E7954F0BD1774B45A9394013317A8925B
:10386000ABB0B4FB5FD737DAC27B9944907F32307C
:103870005CC7E9BE2D2ECF0BABB9EB935FC5C1265C
:10388000D93D2A8C8D23AA8AB920EFC9CEE72CB066
:10389000DF9CAAF88505342BA94E10C5AA74A9F897
:1038A000B0052D43F19C690E5B809060BDB66D63E1
:1038B000E17BFF2887833488A1B2E0C12FBA487426
:1038C000BF5DF05948651518401AFB81B410266198
:1038D000F52E7AE9696B8F4229704929666233397E
:1038E000AE9FEBC3CF388E6607273FFF719E6E9564
:1038F0005F933BA66294C3F9DB2DAAAD7B05E84B31
:10390000AC73B9A79EF674BD439FFBFAD03D7BFA1A
:10391000B686D561B38FBB737EDDE906399D8EF324
:10392000F768C561A9C6F67B75088CF4A27E71AFF5
:10393000443A023D6242CBC4BA0CA90ACBB686BC5B
:10394000EF870D210300B5950F1FBE7C72433E86A5
:103950000D95FA285E6DB93496FF73D6A10F22B08B
:10396000EB8138D34C024A4105646E24F70811BE3E
:103970005207FB1C65CB86EE5A244110A7E8D96A92
:10398000BA86BE2C1608888809D2D6365E2D9D28A8
:103990007750B155B87497C7D14DD20C1EEA129327
:1039A000BE04E8C0841D1E44B9C7566B67891694CF
:1039B00022C8F24F6B4375D713A1DD5E459B26DE0F
:1039C000F3868B82ED6061B2DCA394503289DD71A5
:1039D00087BAA1E157130EBD20A3BCCDB8A678C904
:1039E0004DAEBC70EA73E3B6B6EC9CE6284744677C
:1039F000E401129061A612757E6ABBA204EAB51EAC
:103A00000F9D29A22C4444065767B0917FB6B67328
:103A10005DDF47FC263ECA37E7023695781EBD9526
:103A2000C4E0C176F1FAF58C6AE96BE2E00834672C
:103A3000A2EEE6D672DBC1DA07A5D59C52967F428C
:103A400066E89F4BE80D3C6B721A24F64474C5651A
:103A5000946FD1A1649AB8088BFF658750388A7635
:103A6000488541CA6B0EF21ABC50154233017F1CC7
:103A70006C0B8B058D9DDFBFE647915D0D282FDA1E
:103A80006A044DBEDAE1332A53CE2D3C3A88DFBEBC
:103A900026E87766CD20ED4AD481E0486DEDB75E2B
:103AA0003F76DAD2C714AFC28E01B64C7FBC87C155
:103AB0009EFA2297758DAB88DEA3DB73BFB40674C4
:103AC0009A4313B7B41CBC8E30D99B68963A519276
:103AD000FB4CB0CAD568094AA877BDA1BBA43CC2BB
:103AE0006CB34AE6EABD92DC25FFED6BF125922529
:103AF0003D8E81366881645EC3A68E5A8C7EF6CB7D
:103B0000623CBD13BC67925C58A504A15F0ADD88C6
:103B1000E7249A2C09129AE7A7D79D8A9675D3BCF9
:103B20003A6710CF7D64341BA634328D37C01958E4
:103B3000AEB81C976878A134CEA04525C40D83FC8F
:103B40003BBB3BCF61A5D9B9772DE213A039F47EF9
:103B5000B9A0B26FBC6F95A39E74B60B25FB164A35
:103B60001A8FB649670CA910A2E99B45313973AF8A
:103B7000602B325D92C76FA60A72B123984586CA40
:103B8000A81B23350D36E7648226EEB94B8FC03370
:103B9000C43D9B4A7403C460F252D26657C6A80B58
:103BA000BA8F439359E01973682E5AA38569799B9C
:103BB000199130A3CABE8DAD459A2897177C34ABB6
:103BC0007B9AFDBFAC8C2194DE14332C51B192CE84
:103BD00032CED687AC67A90D95FE5EC11EE33B23AE
:103BE000212B85BDE35290E7E579028693C85719EA
:103BF000DA51E6F15E20F5F23210D1F87BC5444B84
:103C0000684AA769AFEB8D4276087750C934AC2675
:103C1000F1D818B24F92B75DBA64C966A392E7D6DD
:103C2000506A1E3AE329A8F2CDEE60FD0F8C39A749
:103C3000ACBFB3172AA5499E1B11E7095D3C89E774
:103C4000470BD440469C017D1907F1AC14EDC3210C
:103C500022A1CCE7EE3F23F6750DFE974BEF83468E
:103C600020EAFB900B32D0007653BB93FC2E580C0D
:103C7000B551CA6307714512C9756504AAF121D10E
:103C8000CDEF7E6BDB2467807BC5069A799927EAA6
:103C9000E1B0415BAC80A2CE2758AF22A2870A15C3
:103CA000B967A4A7809C69777E41F1F63CBDE963C2
:103CB00052075F2215C63DF848CEA8A2EDF173C4A5
:103CC00079C9FBF1DFDDBAA6C78F21B2AC64AE477C
:103CD000CB10F949DE971C766895FC8A434B0309A3
:103CE000B4B0DF616074D67F28FD7A7A60BBE429C6
:103CF000F92C9B002C6F58F8FBF5642063D1E9F494
:103D0000BF79BD6A4F7D03396111ADFB8479361EE1
:103D100054B871583433B924EC099F085FE10FAFF0
:103D2000E2CFC9168722123298FB5B68CF44FDD3DD
:103D3000AEAD3B884865C5590064795CD7595218C7
:103D40008E9C656A40010A280BA4A9058B0A515B69
:103D50007CE76FF593D678363E18C7CB770A4718BD
:103D6000F763CE499856DA73F18C1E596FA64E99B7
:103D700076F6E4412D14662CDADD50F557C92BD9BF
:103D80009B29C5BB921480D8C03DDE2A35DF98A39D
:103D9000E9A50C0A65D91603AF69A30631340CA74F
:103DA000539B198AAF03BDA47A5A2A3ED3E1A9ECEA
:103DB0004270CD01DC0DF8CFBEA4BAA8420B6C6AEC
:103DC00076EAEADB61F53949453301E7EA5E549C5E
:103DD000A324232C19890F6B72241BB5CE702333B7
:103DE000C4ABE9627E6A26E63807D62D4526D87E22
:103DF000993CB9D23BC44FF125AC5462CF9079497C
:103E0000669540A73613CCC4943E4301AF74EE7957
:103E10006A5E889F5753EF2F4DA9BCDA3EA47C21E0
:103E20005FBBF7E04FCDD602B0A13DAA3790F3D5E6
:103E30001E414F943A2B12E62C85F85A7A042067DB
:103E40006228EC81BE10D1C5A123129005C317B41E
:103E5000FB8ED9E7FBEA542718C998DE5D9F5F0700
:103E6000D36E93FA8EC0B5FB7BF6BB6167FBC508CA
:103E7000DCD32A7F41527E7ED5E2A06979A4848575
:103E80009F9E98B970E334C05A8E563DB189593A15
:103E9000ECDBB809C2287F13FFC033C74083C9DFFA
:103EA000124216937F635CB062C73EB568173A80D2
:103EB000C8D00510368D41A943635A7D301ED28F7C
:103EC00037E1E25EEEBEB0A04AD85466BA82609393
:103ED0009EDD97E625892B711FEC290954A58BAA35
:103EE000ECFAD84BC401D627EEA714F2BB045AEA69
:103EF000A1964EDEC266175FF6F02E953C598D00F6
:103F0000C7BD6027222E473F1B3431F4B6E64E0969
:103F1000C5D4FB56B910396FA8ECE271076F921740
:103F2000EE5E799F56C1112BCB7E3DE020757AE283
:103F30001D3DE23927BA3B81CBADFE6AA0326D9DB3
:103F4000ECF4F4A04CA577434E5942D74F53872A3F
:103F5000CA5F61F2E8C6C5DE4CE884B45719913FE8
:103F6000C2BE8A6607F40CB1CD7AEF09F56142F85A
:103F70000C6E02D74332485ABC559DD36E5A8DB44D
:103F8000755F8CC5A9A553D3B97C5736EA8EC89CFA
:103F90000ECEE0770C0E665DEC8C3A1F742229730E
:103FA000AFB8A4A35DBF09A02516D5FDDCC9A44206
:103FB00063BEE843B58430C0B0E270A65129D8F2A0
:103FC000A7FED8A54339B0FCCBD96C7A5488A0F4AD
:103FD000D794F2B939B3C26E40B6A50D3F02FAEAE2
:103FE0007E29E4B2823FBC2DDB1E827FC60DAC80F1
:103FF000667F0E0F094F3490B8A7A2523F24D6AE69
:1040000008AD886A7B61FBEF07652906FC796512BC
:1040100025E1BB26D6539D3F8DC13A385E974BD3E1
:10402000B4FDF36A89250C9A60A4C3E75008879110
:10403000A79D6D398374B8044088497C057B77441B
:104040001EBFF0BF9573EEFE6E946B64E30BB7DE9C
:10405000103D581A4C382FD97DED8ED0DA0395DCFF
:104060008FE3A33F5D571E1931C3AD7105C857CA11
:104070005303D02BAEF5F63EB81FA28C32697AF905
:1040800058DB7DB2C7A38FFC3E1B8F6763B3F53649
:10409000B3B773BC067E9280EC6BF7F6F75486E3F9
:1040A0003C3A87D2D081AC3DE889FAE9E6EECBDE36
:1040B000D80136E234050E111DD7D09587710F2730
:1040C000C8505C3C92E1EFFBC81E0019A326711892
:1040D00071DF8AD18BCF9619CC7367AB7BE6C2BCFC
:1040E000EA21FEBBDB3B8F198499F9AAC2320DE5A8
:1040F0007846875050D41ABD329FFF402829F6F9E0
:10410000C94EC2AA702BFC3891BE5FCB8A07983289
:10411000A66F0E03C0150A143FE85F461DEE753505
:1041200097FCF4B760B5A9910328A85E074E4B2F02
:10413000358E6190AA3BB08CF255B36E02BAE9D4C9
:1041400081B46E1BB2820CCD36681108FE67454EF5
:104150008ACAAF13F3799DE861F6AAB3281824D967
:10416000511916A46C21A4C95899F5355791359C5D
:10417000B6BC3BE5E9D78E7044FCE7D2535FA8B5E7
:104180001CA65E32F809F6FB213A2D85DFF0DB86AE
:1041900071437B5D4ECB3EC173F1DF5F9B7607EBD6
:1041A000DB3FCDCC733C69FFBB2AE9617D45E02E46
:1041B0008ADAF374A833AD65C671808195E96BF630
:1041C0001D55A1F70B1E0767FADF27677342F943F6
:1041D000A43424AC1FE0191C0DF5AB03DC0C009AD1
:1041E00097A5DA424865141B24EFF4F0F946E5D5AB
:1041F000164549BC08FD2DA5AA2008A00017853446
:104200005490A43EC9EA28463BF22C79A595D1D01A
:104210007E6ABBAF16B4D0EDB1ED5C29A26A08701E
:10422000BD780D29279C32B206D14280F4B7062B07
:10423000FFE95E1005E7C043435F4C61C2AE6661B3
:10424000E27A6EB283A8A88C276DCB0F3AD78F9FE6
:104250008C2AD1067E7105CEE607B3FD0CDF7CB05B
:10426000B84D29AFA19D2CB5B344DDB27FB8EFBBEB
:104270000101DB4EC6D44AC50E851A11E248FAC5C3
:10428000181C9258BA37B5858AE0C93BFA1648CA55
:104290009D27DC22EBDEBE6AFDAA1143C32F6752C5
:1042A000925077A823D6B4D692C2D952041021C511
:1042B00079B288E662FC6963EE7D949588214408B2
:1042C0003432D8E930A591AB0FA1A9BCE6EA56F08B
:1042D000530BF4BAB28EA750D2587CA88D63F93232
:1042E000A136BFEA9CF352F5A34AE2437BE88D99DD
:1042F000A90CE76CBD242E37929486171F3E996552
:10430000D7B61699A529BBED4FFD48294E10C9DB3C
:1043100044A0CC6F927CA0101A6AE08E01DE7EF57C
:10432000A0B1C83BFADBE0F458D90E4DC5660CEDE0
:104330003B698BF56640CF3F4A883A023C129EB8F3
:104340003F1A3A9D0973EA8C89EFF046A623E942A9
:10435000F07ADD63375152A3C7C57565421A95EDF2
:10436000DA8E331D7EAAC033B640FC75E1820701A8
:10437000CE8390697F83E6928674174AB09D1E4B68
:104380005CAFE5C955021ADC3930D686225B787DF0
:104390002C299E65CBFFD4F1F5948F6A5DBFFD1D7E
:1043A000AED2EADAE2C22F199DEADC477CC4A967E3
:1043B0008A16DCE47FFDD4E8143189E6AB46282177
:1043C00060922E24FBCEB091C9C07B96568149F1F4
:1043D000AC2394D89C272B21B215E6ED95100E2125
:1043E000705924FBF4810653298EDB7CE24155BED3
:1043F000DCC3A6D379AD5D1735EA0BCC08C94318E9
:10440000A7C9969A3EC6AB159B2D7998DEFFA6E903
:104410002B27EE71020A318596FBC27CE30608BAAF
:10442000A8C43812EBAA1503A3FDE94BEB1E7EE3EB
:10443000AB67A1584C96FF6DE7D8A347F3EF69F03F
:10444000C0F2BA5C773F99A5237A4647670F0028E8
:10445000AADA864DA5D3C779C8BC9D83E829A2797D
:104460000DF1DAB1807287CA5C15CB91F9EC489AEC
:10447000A7D0DD3EB3F568EFEF0B794FA76AF2B135
:10448000FFA1244D2757B2C7B0BBA6E7469496F1CB
:104490005A14544C0276EE45F78D9E8668188CD4DB
:1044A000E99F32621AD2A641B7635F70C8F79CD405
:1044B00033957CA31AA8858EF8052E86082E4173A5
:1044C000474266BCF40850FA6A2C6B535B042CA17B
:1044D0000844B9A51EF892EE611777E2E77719B69E
:1044E00049A2AFCB30B47FA05A1FCBA8EC691441CE
:1044F000499ED553DC374BB96E44D36B7CC29518BB
:10450000D19284208E2DE38DD34E15A72C4EAE8BE9
:10451000AA272980FE5636DEA318D0F4A6A67D92DF
:1045200081BFF07C63569EB36511DF0AF6D6C5568F
:10453000D6FB9DBDA82E96886320B1BA1E94BA47BB
:10454000CDC2E87CB1533934D0D1EB65A8A85296DE
:10455000358B6C9032AE11FF7E24AF5005AFB06E3C
:10456000B542E06339D4FC1281D606D5F99F2BB44D
:10457000DE58E5CB7FCCADAE46CCA2B08309A0CC53
:104580004A2A7AF370B2691FD504BF757C3CB16CBE
:10459000782F469B5164A8ACB70D748EA5807AF72E
:1045A0005C6D289801CEF5E67E66FE7D984491BC50
:1045B00038F9F5F42A33C3ABBC2A934DF9BEA27E79
:1045C0003BA607E6D219EC2E4E41847F07567A3976
:1045D000DF85F7A52F47327078E4B7DF274BD8384F
:1045E0007C35575ADE688DE29D90AAE004377067EB
:1045F0001DB7CF233DE1ABD6E8739F32B0F88B08EF
:104600001DA4B42805958F018E9EB1D2561141EBA1
:10461000C035AE86E17CED2D92276C857A0BBAEB26
:10462000126B347CB208C8CC4C400C89CC4C21E8CD
:104630000DEDBE9CF2DF99497B9317480E8B58CD48
:104640003A0FCD44C28B143BE5B7085BBD9E8FBECD
:10465000EFB0FED0EDF70C2D5D8973D80C0F790A01
:104660005FD8454D480A7C315EE3E9DDB291813384
:10467000AB100CA6E927A03FE82AFEF9CB2156B0E3
:1046800025EE3E92CA10B6C1BA0AD79C8E80BE3CB7
:10469000F1AF68A4F4B8A51690F4D0CFA16923DADD
:1046A00034466DF21638C71EE31D3FBB39B429846A
:1046B0002D02F4DE92F9324DF714F8DA4A23C1EDF7
:1046C00093FC72E82BE6624A49245EDB21ED480741
:1046D000F8AABDE7F71CF0C0B05B09733A25B1C872
:1046E0008C0F22F2E50641C61CCDC1615DC7EE020A
:1046F00031B2BC51DFA226C24792014758DD345D7A
:10470000851DBDA60B26FA6EB79C9A74259721D3FA
:10471000883FE5355D403A47E49D9FDF1709230B4D
:104720009101B628A12D949BBD53EA6284F9DAF475
:104730002BAB9AD5970120B8D97EB7BCEF2A5990F8
:10474000DAB4A7A41C38F656E01851240E752E8A48
:104750002DFDE432AF60F0AF24653E28D3F43D2C4C
:1047600023B25F0AECEE8262DAB2A2FD6EF0B49A76
:10477000BE382F442A64D7743547EC18616D76E94A
:10478000A8C4B4AD2EC62518BE2B1176B415E82AE0
:104790007F70E6533AEDBFC02D9180EAEB2EBB68E7
:1047A00000A05F2D6AD13184BD9406F4A7199E2321
:1047B000EAB3A24CA0C387F19CADDE4BC64216669D
:1047C000C6CFFBA832765F6A93B3CB1CBA6ACE948D
:1047D000A16D11C8E60A3EF71E589C909BFEB1EEF3
:1047E0008EF40641AF3F284CFAE1B86CC16A7CE117
:1047F00078153564257A4453C34CCC58AC485ED9FF
:104800000889CF15DBD4188198F8540991BEA72FD9
:10481000FC4B2C1391AE4904BFF707FB3ED2C7DD1A
:1048200084FC41EA1871F3E2A5F8C030AA1BC0D499
:10483000F59FC2BBC3E717915D589435FA649BAAF4
:1048400019356C29B92D44DAD1880B2211B1D4E481
:10485000E6E3A9DF7A79ABA7086FCB3C8E54006EF4
:10486000F68719DDEF399F47D0BD8AF0D37E64DC2F
:104870002E18D8D9E7B2492F48B33D12330E7C1514
:104880003C9490730A89511EE49643D9E2759A3B91
:10489000EA7F21620B470B9829277A086A9A894E8A
:1048A0002F688C5EDA452E9D68C074FFCD4E444E55
:1048B00009A2086ACA10FE16C7A619B9873E1BE1ED
:1048C00070AC36FB45465E2F8B826C26AC5239E6C7
:1048D0002E5EA466FC0766DA28CEE11D57B13BE8E0
:1048E000A213573FC76CB54ADCE5E79696FB532BFE
:1048F000AB606C986ED7C32C48AE2EF70F3DF88F87
:10490000A0B20C012EDA00481079C6F70026D2A416
:10491000460B0AAB0D1F8EF312C898C110BD05AE31
:1049200051D18D296AC1D8A21FD97864A7EF8FD53C
:104930006A29D6160EE676E559C63557C9CE17D57B
:10494000B7E8636DC8A85208BC6EE509F80E3C9A3A
:104950004BE4A8C898C4C26E9E7FB0ECDC403E49D0
:10496000E00BCE9E1E0B39014E4F82CE124F162108
:104970006061AFB6D28C3C37319690510FDC90A578
:10498000B13E5F81C3BCC43626F9FE19390F2C5FD6
:10499000B200DC09441AC7C7632C725B658EAFE8AE
:1049A000E14FBB9732ABA6A8F41C4463044FD683F7
:1049B000E4EE4A7AFFF0E53702B51397E7EEE46BD1
:1049C000CF31D5A89061E56537354F8B5D962B517A
:1049D000863ED153B13D418ACDD8E74A0C142D7B98
:1049E000C6B1E111FD35ACB2DE233812870EB3BE7D
:1049F0000F135693D4E0CC9B616862119A75ADA7F2
:104A00000C120D7412F00DC94E0859561611E48F90
:104A1000AD114204A609397F5DB6128302C5B8E420
:104A200036FD4AD0F0D74AD08BC9F2EDF4C42D83BD
:104A3000EAF4190D7E47C077DC7E834087FE7F64F1
:104A4000F2D80C3071E7EC43937E48905A6A63E1E8
:104A50006747DAF07C412DC5E91FFC1AA948A2344A
:104A6000308240FD61CA05DB9556C18BC530DA9AAC
:104A7000DFBC127C88DF9F1A10BBAFE8571DFD21F9
:104A80009B66158AD13DEC8BE0A3EDE65C52ADFD53
:104A9000BEB9DB41006BF398292662688E33463C31
:104AA0000EA399C046A19090B2FDFB6109836C51A1
:104AB00023B74106A4F0075CD95B78367C49F3E460
:104AC00068193FEF151631CF2D08DB9695F3ACFD35
:104AD0007F790261A1763E49641712BD47A53BB9B3
:104AE000283B4EFEA84DAE53116A3C1858DC88771F
:104AF0002049425815F6A1C56786026F48D82F4550
:104B00002C880B2314613F3F9629F002BA237F4F74
:104B1000C99982C0C99C1C63D2FB0EC4DF2F45CD4E
:104B2000E183DB7F81F81A8BA8A372175DBD8EF439
:104B3000C7259507FC597E5F4D307FB1A9BE48C29D
:104B40003F0A3BFB55854E509828D66242ECCAF38B
:104B500022B8D64B9C0B04E1DE28F0634234F8C047
:104B600099F312909AA607C5320FCAC8D199E5CD1C
:104B7000086F4EBD3FC54C76814570DDBD27DB8A91
:104B80007C5C081F5B271B5631926CA75562234D36
:104B90008E9FC0CB4E46FA1DC86987BE69EEC673AC
:104BA000EAB0A79852411C74DBAF2CD7091C5F9B5D
:104BB000FD5D81872314290CE8C99A1C888E8A8A96
:104BC000B60B209B847937CA396AAF9AB39DD21E3F
:104BD000323C07174036E1C58C99095E1680794B47
:104BE00029533A9A3B323B43525B3CC95684D3E04B
:104BF0000923FE5CEA4D0C2AA1F580C7CBBF84BE19
:104C00004F501150FB9119D026A061620946B32381
:104C1000D9D8EFA79692692733E92DFDB03BEEED89
:104C2000C61C90FEFB22DB14E9A44F02E2BA5149F4
:104C300011F22FE44E147C890F23E90A677B74116B
:104C4000C42360F888E49A6CDD8C2D5B38F7F4029D
:104C5000E9379456647938D0CA62B9817C7E137181
:104C60009BFCB0AD99E8370F1FB7A10D828829686A
:104C700030FF4F71A52C67C401810FFA3CADD8B24B
:104C8000CC6DE308D0778F480F014A40ED1617B777
:104C9000DB819DE2624FF2071A22CCF942B4C701D0
:104CA0006B78AD274068EC941BDB9185ADC561A79F
:104CB00037D61BA5944576A1AD99DA9ADAB8EA5FA2
:104CC0006A8C046F4DECF4BD63BA8A8AD126BC0F9E
:104CD0002C10ABE5C7441FE09A88BF7620DAA58286
:104CE000C12991041E064F9241ACA4F1DE93E6D394
:104CF00067B428A46CDBED98E6B69E387F8CA6DD01
:104D00001C931F9106808D829D33307BAAC3231490
:104D10004E06D39EB5A6240575AEBB8ED2A40F7DDC
:104D2000C1FB2631013A54A2E8EFDD20B116DD0CBB
:104D300022100E2C44CEAC4E1BC069875EF85D700D
:104D4000384A4DDD719FFA11E8ECECAC82AB5EB7EE
:104D5000F764EF45A509242A55B463CF971DF0AB3E
:104D60004B3056656F6A11EBA3A3D47FC186E33045
:104D70005C0DF77692E8B70D0E04EA44FE0AB7F927
:104D80001AD868C85E8FF7C578C975EE9EA17DFFF9
:104D9000826DCAD01A0092B7809403B0C92D2F68D3
:104DA000A868F91ACB1E023EE824DBC862C878DF87
:104DB000372FE2972D1D5286CEC18525F0E79A1137
:104DC000A84EA85408F463ABAF973852C4E7C8C7DD
:104DD000FE333D3176C48123AFB2024059CC054A3F
:104DE00002FA46251A1A6579B70313C67BF2E8FE64
:104DF000CD925444308A46FADB7D63EF0602DE042E
:104E00008098A6532A29777E1EA8A276351782F8A5
:104E1000A585C0ABE0B45FB285A20CEB963D31979F
:104E200062116512DDD44DBE6B612D3876BFE8008E
:104E30005437E991852C631DBEB30589EF5ABECA6C
:104E4000C48782E146F1AD3AEBB7A6F2D60838C77F
:104E500079AE6B632DFB344AEF824EFCD9A04968D2
:104E6000CC5F2E870AF0C9F52C67DE19EA2D8F1763
:104E70005B2376EC3AF209D28A599FCF478A73D6E0
:104E80001631FEAE4BF921CEFBC895716F71ABD5D3
:104E900064988A5EF952CDE9140C9C38AF43741AB9
:104EA000E9D2049C8656C7E68CEEE2225618972873
:104EB0006A0D39DB4427448B4E3253E2CE9576C5DA
:104EC0008F456E0719D67E122524E8F3D908818F05
:104ED000BD663E1066CF3612367D7DDD316448FCFE
:104EE000F921E33D85A8543D2800DBE01C0981D56C
:104EF000F1D1932F1E051CAC9A653B3295F959E20E
:104F0000BEFE9E569BE5A74DF9C670D19234C38173
:104F10002EA3877C522CEC17DBD479081E646571B4
:104F2000C1D58B2E1A11FD4A91FA67CB622D20173D
:104F30009AB47094E150C03638014D6A66B533E6D4
:104F40007BFF92146A11A34B2A61FDE66D8D1195CA
:104F5000AF40119FCDB3BA1C593350673907C6E62D
:104F60008D97943175C769B42DFA2CF2E2413A332A
:104F7000CD4564AD90E7BBC224FB60701AAFFF4C17
:104F80000ED1C5D756652C79597740EC5D10D49574
:104F90004788BACECD85286EBD409B6BADB1CE9A09
:104FA00035CBB95ED4B39D69712FAFC58E08CCDD0A
:104FB0006D6F2BF7CB818070FA294385C15B330B72
:104FC00081F5404B3F5779C582421F8063AA56B393
:104FD00060898410749964A2322D87119444A56469
:104FE00044E41306242A3211A169DCFE400DA4B466
:104FF0007705D18742A4FAFE118BA93E4A5D1A06B5
:105000002B52616DD34A4C46D789624F76DE8BAF07
:10501000C8451017578E9C0CBD51922C447D9B4F58
:1050200032C82CB5375134362D6A54778515C7E40C
:105030001E31E06443BB2D3C80B6DDB21BFDD7457D
:10504000DC09B78CB8819D122DA222BB463CF845E5
:10505000CA6A133C337C3500F447E38DE973D8E822
:10506000C1CF0FF160A6C7F733DFE912CC55B323E8
:105070009984F35F0F157F8B16059518791E764579
:1050800086D6A04558254699DC70D6B948F10FBBA5
:10509000CB3FC5974BA7F9E4527AA89DCF3CE48358
:1050A0001DBD3D470FBDB0960D3FEB5241E279F07B
:1050B000DE933C3685F37A7020454A535CD7323014
:1050C000F300A7CCBE1339DAE149CF24B16924D467
:1050D00065B4B44F77F72BC2892E53AAB81A373A62
:1050E00006C79D99EBBE1DE120D8F1AB0E3BB8740D
:1050F00049326B4370D451CDA7F328D6F735380F1A
:105100003E3F60203B9A6E0753FDFDA38CBD55AE1C
:105110000C6C63FC87E8D57FD6364F46AC75A7127A
:10512000A700BEE388F40D938B6138A104785A324E
:105130002F720E98879DC866064ED329E34A6BFAF4
:105140007247C46146133B67767C62092C554896CA
:105150001957C6BDBE053809750F3588226F9D8168
:105160000DBB16818E32568EF40C6C3579752D5828
:10517000ED317C70510CEAA7CBFF9DC2023E461870
:10518000DE6FB468141F64D1F7FCBE779D8E44FBBC
:10519000DC6EEE109A350720450BB1193D2AABACF9
:1051A0003DEC8D463E389E531F2472793B363C7D44
:1051B000F34161E50FDED4FBF2AD4CDBE19364B566
:1051C000649C1D2A4076131E8762E0B6B42583A432
:1051D000A40921C6FECC4599053B9206A0D1C97809
:1051E0006DDFDB1B500338195534AF554D841D4519
:1051F000C87A919CD0E28133FCE4CA7A977C67E656
:10520000C0C24937743D680B2B7B4B1987D808C641
:1052100029BA09565E242102DC0B8CCF0CFBE02E50
:10522000710724149AECD93E374812CCEB3A24BDCE
:10523000394306BD37E5065FD4FCA4BA2EDB12D095
:10524000E6CEB5A5D797882034F000997E7BAA6F6B
:105250008620AE2C426A6268831930E45D6BFF26BB
:10526000527AB4E99E7A492902113ECBB6FA4C80B3
:10527000BE192B54778C58147411495A3D01404F74
:10528000C19EE86B06D299EC081848F3C6A17D08C8
:10529000E9E78B80145BAD9B4C95CA85C3B738D9C1
:1052A000E320C8185D46EC9302D3F9FBE6D69501DE
:1052B00019071F26DAE00E762ADE56EFA77742E7B7
:1052C000843C0E7E39AF03E73C491AEC2E40EAB726
:1052D000B1E401FE71172D1ED017712A4177FFBE70
:1052E000A96CB8F33353AA9B2DDFA58CFA23D87E83
:1052F00083A210F8ECB93EF1590DB137FE80386B3E
:105300009B7A9857F90EAF90CC849FDF1D8E5EBCC0
:10531000F36710881277BCA4B6398292DED3CBBC77
:10532000253E7A47DFC4E66BA61CF9B9B286C935BB
:10533000AB3279973E5862FF2EF1362D3D35D3AD15
:1053400083C980689DD6EC8D77F8ADB4022F7DA11E
:1053500085E988E84C580600C28FED2B163AC389C0
:10536000961DCEC527D3FE62891E73F3BC513DAD99
:10537000A18E0D1EDEF4CCC9D023532F9EC604DDB2
:10538000E5B9A14E276FE8651AE068EC80D3F937DC
:10539000C02079F2471791503164EF03EDBDF92C2D
:1053A000E89E5FEB08173794B20AD6532CF9459C58
:1053B000E3E49FA6BACC048BA6B0892B92A31A4E25
:1053C000B36F4342C082CE4810F7C2B517E30F2631
:1053D000D29CDBA7B9989DC6E54A0F1192CB4C74BD
:1053E00085B85DC7FA9C887ADB244A0994065FE891
:1053F0001FCF3D27360480CF2D628DFA7C173233C4
:10540000A641BFF7C55BAE18AE20DB525FC9302D99
:10541000953F7047576DE512969ED51C27DE99D2B1
:105420008D3E4D5C20B5A587A2567173D007E0ACC8
:1054300089C343BD561C2563A87C9F6CD52C76DAA6
:105440008E25BC62FACB694B1C0E1E830387217F1D
:10545000569FA535CEA9BFA1FF055A61AE47B181C0
:10546000967023CDBB43F3E76752DCAA5A85F1FB64
:10547000D589B126738712754B27F0492B2B80A451
:105480002046A0E337BCF134DD55BAF8491DFCAA2B
:10549000F89D316DC7747A89DC1251FAB0325760C9
:1054A0006AB078C762CE0D3C36307349B05B9E94CB
:1054B000079ACA47715ADD647776610BA36565CF99
:1054C000FBCDC42A3D34E4D5CB2A6A122C08D5AED4
:1054D000A7A8DA94B64C517D974234B9EC9F33A615
:1054E0007D9E7B55CFB52BC833C24C24ABF542CE45
:1054F000EE72AEFCCC2B4AB12D8973E7B940D92BA3
:1055000025D5FBB4F4CEC30FD5908FBC5F9F08D9CF
:1055100031D510B46B51873FB6D8283A238F9E39C6
:10552000964213915AF28449375FBEEB6AD4DDCDBF
:105530003EA416488AA8039036F79561814A171B46
:10554000ECFB2F9D6B099416AFA112B4FDFF89D817
:105550009C75059A164BA45324E6050C7CBBD550CC
:1055600089EA30B6D354D0A93D1EA7C55F2512BA2B
:10557000ABF320CCEA7BCD4AE79344FA780D49EDB2
:10558000EF979E658CE8B49D80F2819C2C93DD831F
:10559000184EB34F6C88B96EA459E43978BFBD5525
:1055A00061D94186F6BACD1C01BA37A67E80D5E115
:1055B00011971919B109EE391779A7A524A5880003
:1055C000DA4609729E78C49BE6B5BE5ADA37F57B97
:1055D0009655F6F826E2558A5E37E6A4681A46FB29
:1055E000CCA41F1A245B15C373C97BED38291ED9BF
:1055F00087696EAB99EAC091FBF4B13B732FC1F29E
:1056000074CF8B4CAA73A5CBC96877F1736DFB3946
:10561000B557CB48E6EB68CAFBFE24B8E2AFA40F4F
:1056200034283F325BAB69ECD0A625884EEC3BFEBC
:10563000E6535602E5B47A11C483A485ED8BFED1FE
:105640001B2091DE9DD4AC48D873013C6DF607FD5C
:105650002F971170324C220B026BD4408DEB975474
:10566000357FA6B1CA7EDFA3CF91069BFC0FB66142
:105670008D0B0C8DD06E0DF9BF9984F22BBD9F99C7
:10568000A775074D54EC323396E5A01D16C2D80C11
:105690005FCBDC49A21593CF3D604EB9B50CE2F566
:1056A000485D1DEB2D9D5E7F38090322327EA73BAE
:1056B000D140205CE5A81E07AE11107D42CB9FD7DC
:1056C000504964855A32B716AE2000D5BAA9B7C979
:1056D00006F64502DC2E79A961749E2962988F93A3
:1056E00024576F12CA4FD96D5A8F97847036C6E906
:1056F000293FB39B022A5D7A35D3096DA38D45AA54
:10570000C79238D16BE226D10CACBE95CF85E26949
:105710000C6A66642C42A6B855381896D04ABC501C
:105720006CAAA6FA7487D1A584B3D166051FA862B6
:10573000B64649E642EF8874385EF740476E9A47AE
:10574000328B69C1CB38D884AF4E8DB91CED7D3515
:105750007739ED5B26969886017BA31A8ADD7CA1BA
:105760008EF645AD690FC5BA1F417A2CD356F5A701
:10577000A9602C43F4E8464BCB74C5F6F12C2D966A
:1057800031ABC1B4545A305705463434A776E8805B
:10579000B5C72F81ADAE60F99A548D3BF3ED584DEE
:1057A0009B7F77B159F7398A4FB5F5F63644875262
:1057B000C308AB3578A2AF952DC2064CCBFA5E116B
:1057C000C897E38891D7A4965FE85B3267DADB4C31
:1057D00048BEB7B35127F116D468FA1745775C264F
:1057E000FD77954C46163824F4768C8E0045186E5D
:1057F000F1C669304C16474C656CE783C53A971B78
:1058000015E04A7C635729CC5D401E5822FB2AE8EC
:10581000C35E0C947B7D320F56786A214FFDC32006
:10582000DADECA664B657D8C3ABAE7F24498B05D21
:1058300016C4335B3E8E91B67005009D1BC33C2899
:10584000C36F940E192827DA38B617A6A9275AA6C7
:105850003AD57E0CB4CCB5997CFC0869233A00910A
:10586000F30A8FBFD42C40478C58AEA83EF9AD73D5
:10587000ED4D0C00616D23BD10982A517ED780B389
:1058800058B749E445C3D829BD25DDDF4DC580752E
:1058900072DDF4EC8F6A6C299EDEA484E82B534100
:1058A00083EA090056C47E668030B8D812EF7FB80C
:1058B000E8B18D935509D53752922C412FCA64FC1B
:1058C000733F50356748EA95EC77C74C3F583781AE
:1058D0001B989EF70621302F59EA5762347B10A59A
:1058E0000B9EA49054803EC2A64577E00F3BCF5755
:1058F0005641B045F79892F0E04A44618FD0D9AF55
:105900000486E54C016B4EF837AB15C1C5DC8961E7
:10591000E4F5F8ECC44FD762A74D466AEFCF639C1D
:105920002F3FB7E1D8002D3BA086BC809732BAD973
:1059300029DE504F81488A3036CC52DA69B35CC5D3
:105940004B73F8487793C74AB5483DEC783C3B1712
:10595000E50B6D29F3D38F3A725C4B960976CF40F5
:10596000B961093109CD428439AD3DC7F15747DFEF
:1059700008579E6FE1FAA050A99CE1DA08308F6EBB
:10598000A8AF82E28A277D12D266B8EEF62FCD3B11
:105990008F8DD6DEE95762E2B3623BF475B7767F4E
:1059A00004C894439DD87B83A989B75AF40D8553C5
:1059B0000EFB1D388FC999B73FB8F42FC05CD14199
:1059C0004C57E5C9ECEA18D6BC84F01DBB753F7294
:1059D00076E7CCFEAE03DAE792717821F8424DDE2D
:1059E00008AF5AA75B4434CA80EB2D200F804926AC
:1059F00068DB738BFCCDB887E40BAD3622B7108A19
:105A0000E8A57700B58FC63AE8FD3B5F1B571894B1
:105A1000D553A8F944B4565C5FBCCD42F0CEB9B7BB
:105A2000B4271453D05AD9D283E0E81A6E8A934827
:105A300041BC24BA6C8380F2993E797AE280D17EAF
:105A400021D23ACF1FEEE9D46A6FEF21F0B87B0C78
:105A500002EEBF09079EBD401833179C46998CE0A3
:105A60004929E786F0BC8ED121BBE65F3D7C53FF20
:105A70003722700B35207F4BAFA680D80576DE220B
:105A8000D6FC002B1B7FB79A964442C65EADEA5FF8
:105A9000DB74199AF7476065F6E5D2D121FBFFE583
:105AA0005B5F9982636C7D550931859C85DB94D55C
:105AB000882219361EC165B2E8B4F0F8C80B7AC75F
:105AC0007F09E1390A4DA0AAC1403EFA2BEED73D2D
:105AD0006C7D0717ECE9B63358EFC7B42583E9129C
:105AE000CA1578BB26C5AE2C95CE9CA933847B7392
:105AF0009CE05A738D265794EDB54617881986E7B2
:105B00002ABCDD77DB0528CBC9B2075306508FCA04
:105B10005C5586532B6B73007BED3EA0027606CC62
:105B2000E9705033392785DDCB1F5519EFF28A58BC
:105B3000348532617DAC5BC412DAD62973AB59B2BD
:105B4000CFDE5B3778339695105EE246AB8144B189
:105B500073AD1C436E9CF6557DFA71256304382B9A
:105B600074F4C999746B285F104B5E6FE09A89DBFF
:105B7000411E36FF7226F3838B85FB6B2086E1E6A0
:105B800097B6CEAFC37F38747AA4FC210A78B64B9F
:105B90002E04C66171972A9EA417620D6EC5CAD8DD
:105BA000F2317C77257C60FF574E5C4C3C324FB223
:105BB00020F41970B2645E89FA14B5CEB3DDE6162E
:105BC0003FC6B9606F73E7DCCB94DBA480B3BF51F1
:105BD0005206FE46C1F16A9C632B21BDBC4D476E47
:105BE00045A7EBD6C587309BB214392C35692EA456
:105BF0006ED4BAE246D7CA28D456488EAEDFC81152
:105C00008FC8A7F67500A149A4B34A4184AAA3E6A8
:105C100067A641F3C413BD1AF9C301F2068797EFD3
:105C2000BDF8DAE4BE0BD5CA0A19603FA42D195598
:105C300088F73F15E8D1022D1B9340402048486269
:105C4000775AA2C232B258582EB132862A03C10105
:105C50007FDE3D048F2FB8A532BFC6B58FAB4ACECD
:105C6000BAA1FBF76F2F8495BF2EF43C3186D86B19
:105C7000897561491ECCDF085C1C79319C9910AF95
:105C800096D022FF0703E2612D35F8CE46AF3C0FD8
:105C90000EF9E3D4BF85524E61586582849165E266
:105CA0008DA5482433331296947EE1EB90AA1EE032
:105CB000C39487FC0BFA288B01972FD2ACCC730CC2
:105CC0008E24BDF1074D3A7FF3DC03A1B81B0F9979
:105CD000CE364C6C1287F4A1B698139B83AAD3AB33
:105CE000A17C68129A54FAE8A82A1A3D94BCB4150B
:105CF000F651D16AE4A01DA714B92DB37A4DC07333
:105D00005C6F0FD049CEF0672B0E4DAD0E189F067D
:105D1000C0DA7FBB25F82F4FA06C0AA9D5AB00488D
:105D2000F3FC919B0658CB2A6976BD74F984984B95
:105D30002AC4F7B2E1904CA489492CC3C7195AEA86
:105D4000A8E9CD9F626E53EC6CB6E138CACF7715E7
:105D50005EDC13759F307F2D436844D9E716954567
:105D6000219A974264D14A041191AEA1A6FFD40BA7
:105D70000E594CDC85DCB9EE410E91AED8E70BCB69
:105D80004F007997CAD66F9739011E5CD92F017AD7
:105D9000134808E2D3FB8FE834A7C056B06BDE5936
:105DA0002105562B25DC60F2ADE7238C90B6CB9015
:105DB00044EA4962F2105F40BB25FB8B5914FFD8BF
:105DC000C92438E878DC7100C41321C056A5BE563A
:105DD0005757C0E4478226E83077251CF5F0352F69
:105DE0005B29492F7496B58478114065C9FE4BBB79
:105DF000A71FC88E23803446942AE165A811336C0E
:105E0000DC65DA1433066B04D33D3FB94A747F4234
:105E1000322682A645F96E9B5DED4934C3477C6509
:105E2000332F3D852F1FE3DD6E1EF24701B7BDB353
:105E30000C54C2424CB9DFD3B792A7FB8FCC446A53
:105E4000A653D6133F59997058563A7F6193678D80
:105E5000A6A78342C9A79D4E7E38F62F27C13A8F49
:105E6000E0B2619689F5CD34188D4434CD7D3BCEBA
:105E7000567ADA1D21A81DF0DCA38A352C94E49E05
:105E8000BACB562222D33CF316B58AE0247D5C625D
:105E9000A597D4C820C46E1DBDCA779293D34D5424
:105EA00049C37952C2017A02433C20C6C8C089BAAC
:105EB000829F3A11F771B0B4125CB0089317744D19
:105EC0001787B0F4F0964AC31A665B429CB457EB4E
:105ED000E46DB6F79F30D6B3FEF861117CC5BB996F
:105EE00015B90C4ED1BACCBFF34EB6CF24BD1AEEC5
:105EF0001F19A6E6A388F4A3EE6D3965A5FDF5F09C
:105F00002810772335393D9676B0B395B26AB9D467
:105F1000BBF2F1E5F935B1FA774A943C2765BD94B7
:105F2000462C4BE4EA0F90319FD8C465CAFD8E4FD2
:105F3000899FF73DD916F43CBB72D58FCE227DEEFA
:105F4000F9888B644D1E8B4047F9C9AC5FD5713819
:105F5000AB737B53D91D2364E5F4275B7F2CD88F6B
:105F6000DC3B0E70B5C9CB7EE1E768854E6A5266B0
:105F7000E21E974042EEA5B62518B7141F1EB0606A
:105F800002FC2B3D13E7720D5EC985758FBFE936A4
:105F9000D6EF384D35035F469A43E69F9A28C26C88
:105FA0000D5E2880510266A246C7C80930BC49A8C8
:105FB000C54B0413FE372C26FB0DDD6778BF25B8D3
:105FC000508B629B565F36B0B7B9731FADF55FDB80
:105FD000A32691F4C926485EF15BD8AD73EA586AEE
:105FE000106D9EDC283A1408FA4D45AB3984E21155
:105FF000655D0FB41E3D2B258682C0FF9CD8FCD06A
:00000001FF
